:06000000020030020117AE
:030013000200C127
:01001B0032B2
:0300230002017F58
:10003000758150C2AFC2B4C2B5D202C203753804D2
:1000400012042590009D75320812044B7532081277
:10005000044B7F641201D89000AF75320812044B34
:1000600075320812044B7F641201D875891075B877
:10007000057598D07530057531E11201E71204D588
:1000800075348675352D1204D51201E7758D00750E
:100090008B0075A89DD28E75870102009200207793
:1000A00077772E656D67406F6C612E637A20200034
:1000B0002020656D676F4069406F6C2E637A202049
:1000C00020C2AF7F3230031CE53870037538091544
:1000D0003890016DE5382393F536E538230493F520
:1000E00035020106E535B42D0EE534B4000975344A
:1000F000A075352D020106E534C39401F534500690
:10010000E5359400F5351201E71201D830B303D27A
:10011000AF327F050200C5C2AF7F3230031DE53824
:10012000B408037538FF053890016DE5382393F561
:1001300036E538230493F535020106E535B42D0E76
:10014000E534B4A00975340075352D02015CE53441
:100150002401F5345006E5353400F5351201E71277
:1001600001D830B203D2AF327F0502011B6E087294
:100170000876087A087E08820886088A088E08C2EF
:10018000AF7F141201D830B0FD200308D2039001D4
:10019000C6020199C2039001B475320812044B756E
:1001A000320812044B7F641201D81201E7C298D2C0
:1001B0009CD2AF220056737475706E6920406B6DCF
:1001C00069742E202020005679737475706E694012
:1001D000206B6D69742E2020C2AF7E0D7D7FDDFE09
:1001E000DEFADFF6D2AF22C2AF85343C85353D75ED
:1001F0003E00753F008536408537417542007543A6
:10020000001202DB853C30853D31C200C2B4C2B76A
:10021000C2B5D2B57A02783212023318E67B08C230
:10022000B7335002D2B7120233DBF4DAEEC2B5D2E2
:1002300000C2B7D2B4000000000000C2B420000128
:1002400022120247D2AF22C007C006C0051204DD49
:10025000200305783402025A783612027312029390
:1002600075330075320812046012030DD005D006F4
:10027000D00722E675F07DA4F53CA9F075F07D0865
:10028000E6A4FAABF0E9C32AF53DEB3400F53E7580
:100290003F00229002BF7C07793478437A04E493CC
:1002A000F6A318DAF91202DB073001F9173002055C
:1002B000C3E72430F709BC0503772E09DCDC2200F4
:1002C0000F4240000186A000002710000003E80054
:1002D0000000640000000A00000001C0D0C2D4D2B7
:1002E000D3C201784079447A05DA030202F718197B
:1002F000E6C397401360F2783C79407B04C3E697ED
:10030000F60809DBF9D0D022D20102030590034F91
:1003100075320312044B200307900353AC347B2146
:100320009003F87B09AC36E493B50303020340A3C2
:10033000A3A3A3A3DBF190034A75320412044B225A
:10034000753203A312044B02033640204D487A4510
:1003500020202008455338200A455339200C4553A6
:1003600031300E455331311045533132124553313E
:10037000331445533134164553313518455331360E
:100380001A455331371C455331381E4553313920F6
:1003900045533230224553323124455332322645BB
:1003A000533233284552302029455230782A45525D
:1003B00031202B455231782C455232202D45523276
:1003C000782E455233202F45523378304552342011
:1003D00031455234783245523520334552357834E0
:1003E0004552362035455236783645523720374506
:1003F00052377838455238206E454B322072454B83
:10040000362076454B31307A454B31347E454B3181
:100410003882454B323286454B32378A454B333230
:100420008E454B3337C2B7C2B1C2B47F021201D876
:10043000753206900445E4931204A97F011201D895
:10044000A3D532F2223332280C0601C2B70532E4BA
:100450009344801204A9120496A3E493D532F422A3
:100460001204E778330532C374089533500CE53332
:10047000C394082440790002047FF909E64480C24D
:10048000B71204A912049608E6D90705327440C2CF
:10049000B718D532EC22C2B7D2B4D2B1E5905480AD
:1004A000C2B170F6C2B4D2B722F5F07D0254F0FEAC
:1004B00074FF540F4EF590D2B17F1FDFFEC2B1C55D
:1004C000F0C4DDE922C2B7741C1204A922C2B774B9
:1004D000181204A922C2B774011204A92278337930
:1004E00009760008D9FB227834A93219E6C3943082
:0904F000600122762008D9F422F3
:00000001FF
